:10045200B1B2B4B8C3C5C6C9999A9CA3A5A6A9ACA2
:10046200171B1D1E272B2D2E4D4E5356595A5C63BA
:100472006566696A6C717274333536393A3C474B3A
:1004820078878B8D8E939596CACCD1D2D4D8E1E25F
:10042400C101C102C180044D000000000227000088
:10043400025C0000025E0000012A00014C00014B36
:0D044400000121000122000423000000003F
:10001D00EF5403FE25E0FF4307F9D294C294E4FDAB
:10002D00C295EFA2E39296D29525E0FF0DBD04F0A7
:10003D00D296C295E4FDEB25E0FBEA33FAA296E4F5
:10004D00334203E4D295C2950DBD0DEA53020FD292
:06005D0094AE02AF032285
:10006300E54BC3942050F9AE4C054C742B2EF8A6E7
:0700730007534C1F054B224F
:10007A008B0C8A0D890E8C0F8D10E4FFFEF513ADE3
:10008A0013ED3395E0FCC3ED9510E50F6480F8ECB1
:10009A00648098501AAB0CAA0DA90EED3395E08D29
:1000AA0082F583B11EFD2FFFED6206051380D0ABEA
:1000BA000CAA0DA90E0510E510AC0F7002050F145D
:1000CA00F5828C83EFB14B0510E510AC0F70020579
:1000DA000F14F5828C83EEB14BE51290045293FF14
:1000EA001163E51090045093FF1163E4F513AF1305
:1000FA00EF3395E0FEC3EF9510E50F6480F8EE64E8
:10010A008098400221E0AB0CAA0DA90EEF3395E0CE
:10011A008F82F583B11E543F90045293FF1163E519
:10012A0013FD3395E0FCED2401FFE43CAB0CAA0D72
:10013A00A90E8F82F583B11E540F75F004A4FF8DAA
:10014A00828C83B11E54C0FDC413135403FDE5F021
:10015A00EF4D2452F582E5F03404F583E493FF1160
:10016A0063E513FD3395E0FCED2402FFE43CAB0CA0
:10017A00AA0DA90E8F82F583B11E540375F010A43F
:10018A00FFED2401FDE43C8D82F583B11E54F0FDA0
:10019A00C4540FFDE5F0EF4D2452F582E5F0340426
:1001AA00F583E493FF1163AF13EF3395E0FEEF2479
:1001BA0002FFE43EAB0CAA0DA90E8F82F583B11E95
:1001CA0054FCFF1313543F90045293FF11637403BA
:0701DA002513F51301F822C3
:02000B0021E1F1
:1001E100C0E0C0D0C000C007A20192B0E4F5212058
:1001F1000208E54B7004C201804320020CE54BD399
:1002010094004005D202752908E529C394084020CD
:10021100E54BD394004015AF2A052A742B2FF8E63D
:10022100F551532A1F154BE4F5298004C202800DB4
:10023100E551139201E551C313F5510529D007D0BA
:0602410000D0D0D0E03235
:02001B0041475B
:10024700C0E0C0F0C083C082C0D0C000C001C002FF
:10025700C003C004C005C006C0077F02111DC00649
:10026700C0077F03111DAC06AD07D007D006C3ED4D
:100277009FFFEC9ECF255FCF355EFE7C007D0AB1E8
:100287006D7D12B1818E278F28EE3395E0FDFCE559
:10029700262FF526E5253EF525E5243DF524E5231E
:1002A7003CF523EE3395E0FDFC7B007A307900784E
:1002B70000B1B77B107A2779007800F129E5502F34
:1002C700F550E54F3EF54FE54E3DF54EE54D3CF516
:1002D7004DAF220522C3EF6480949E4024E4F522AB
:1002E700D2007B1EFAF9F8AF26AE25AD24AC23F178
:1002F700298E5C8F5D752600752500752400752392
:1003070000D007D006D005D004D003D002D001D04A
:0C03170000D0D0D082D083D0F0D0E032F3
:10032300759852758902758DFD758C06D28CD28EA7
:1003330075A88A75B802E4F50AF50BE4F508F50922
:100343000509E50970020508E509B430F3E508B4C9
:1003530075EE7F03111D8E088F097F02111DC3EFF8
:100363009509F55FEE9508F55E050BE50B70020543
:100373000AC3E50B9408E50A6480948040BD20001D
:100383000543870180F8C200D297E4F508F5097F99
:100393005511630509E50970020508C3E5099408C9
:1003A300E5086480948040E77F0F1163E55CF553B3
:1003B300E55DF5547B107A0E79007800AF50AE4FAF
:1003C300AD4EAC4DF1298E088F09EEF555E509F5D3
:1003D30056E59054FC4403F5527B007A0079527D34
:1003E300057C00751100751201117A7F551163E5C3
:1003F3004B70FC2002FDC2972092837F03111D8E58
:10040300088F097F02111DC3EF9509F55FEE95086B
:10041300F55E755000754F00754E00754D00618196
:0104230022B6
:0300000002049265
:0C049200787FE4F6D8FD75815F0204D984
:10051E00BB010CE58229F582E5833AF583E0225092
:10052E0006E92582F8E622BBFE06E92582F8E222DC
:0D053E00E58229F582E5833AF583E49322F6
:10054B00F8BB010DE58229F582E5833AF583E8F0E6
:10055B00225006E92582C8F622BBFE05E92582C892
:02056B00F2227A
:10056D00EFF88DF0A4FFEDC5F0CEA42EFEEC88F0D3
:04057D00A42EFE2288
:10058100C2D5EC30E709B2D5E4C39DFDE49CFCEE95
:1005910030E715B2D5E4C39FFFE49EFE120606C301
:1005A100E49DFDE49CFC800312060630D507C3E4FC
:0605B1009FFFE49EFE2204
:1005B700E88FF0A4CC8BF0A42CFCE98EF0A42CFCE3
:1005C7008AF0EDA42CFCEA8EF0A4CDA8F08BF0A461
:1005D7002DCC3825F0FDE98FF0A42CCD35F0FCEBC0
:1005E7008EF0A4FEA9F0EB8FF0A4CFC5F02ECD3985
:0F05F700FEE43CFCEAA42DCE35F0FDE43CFC22F2
:10072900C2D5E830E70FB2D5E4C39BFBE49AFAE4FB
:1007390099F9E498F8EC30E717B2D512075F120679
:1007490097E4C39BFBE49AFAE499F9E498F88003E7
:1007590012069730D50DE4C39FFFE49EFEE49DFD8C
:04076900E49CFC22EE
:10049E00020323E493A3F8E493A34003F68001F24E
:1004AE0008DFF48029E493A3F85407240CC8C3335F
:1004BE00C4540F4420C8834004F456800146F6DF2E
:1004CE00E4800B0102040810204080900424E47E96
:1004DE00019360BCA3FF543F30E509541FFEE49323
:1004EE00A360010ECF54C025E060A840B8E493A3EA
:1004FE00FAE493A3F8E493A3C8C582C8CAC583CA15
:10050E00F0A3C8C582C8CAC583CADFE9DEE780BECC
:0104510000AA
:10060600BC000BBE0029EF8DF084FFADF022E4CCD8
:10061600F875F008EF2FFFEE33FEEC33FCEE9DECA1
:10062600984005FCEE9DFE0FD5F0E9E4CEFD22EDE7
:10063600F8F5F0EE8420D21CFEADF075F008EF2F31
:10064600FFED33FD4007985006D5F0F222C398FD22
:050656000FD5F0EA22BF
:10065B0075F008758200EF2FFFEE33FECD33CDCC56
:10066B0033CCC58233C5829BED9AEC99E5829840D9
:10067B000CF582EE9BFEED9AFDEC99FC0FD5F0D6B6
:10068B00E4CEFBE4CDFAE4CCF9A88222B800C1B9E0
:10069B000059BA002DEC8BF084CFCECDFCE5F0CB1E
:1006AB00F97818EF2FFFEE33FEED33FDEC33FCEB57
:1006BB0033FB10D703994004EB99FB0FD8E5E4F912
:1006CB00FA227818EF2FFFEE33FEED33FDEC33FCFF
:1006DB00C933C910D7059BE99A4007EC9BFCE99AF3
:1006EB00F90FD8E0E4C9FAE4CCFB2275F010EF2F38
:1006FB00FFEE33FEED33FDCC33CCC833C810D70738
:10070B009BEC9AE899400AED9BFDEC9AFCE899F872
:0E071B000FD5F0DAE4CDFBE4CCFAE4C8F92205
:00000001FF
